:020000040000FA
:020000003F2A95
:08000800F100030EF000831665
:1000100003138C1E0F28831203138C1A18288316BF
:1000200003130C1E1728831203130C1A2C2A3A2AC6
:1000300083120313F60A1A08F20001307602031D38
:1000400024287208F300252A02307602031D2B288B
:100050007208F400252A7208F500F6010514F7016C
:10006000F31A4928731A5B28F3196D2873197F282E
:10007000F31891287318A328F41BB528741BC728FC
:10008000F41AD928741AEB28F419FD2874190F29C9
:100090002129731AF715731EF711F3197715F31D3C
:1000A00077117319F714731DF710F3187714F31CF5
:1000B00077105F223329F319F715F31DF711731920
:1000C0007715731D7711F318F714F31CF7107318D5
:1000D0007714731C77105F223A297319F715731D73
:1000E000F711F3187715F31C77117318F714731CB5
:1000F000F710F41B7714F41F77105F224129F318CF
:10010000F715F31CF71173187715731C7711F41B8F
:10011000F714F41FF710741B7714741F77105F2205
:1001200048297318F715731CF711F41B7715F41F82
:100130007711741BF714741FF710F41A7714F41E58
:1001400077105F224F29F41BF715F41FF711741B6A
:100150007715741F7711F41AF714F41EF710741A38
:100160007714741E77105F225629741BF715741FBD
:10017000F711F41A7715F41E7711741AF714741E18
:10018000F710F4197714F41D77105F225D29F41A23
:10019000F715F41EF711741A7715741E7711F419F8
:1001A000F714F41DF71074197714741D77105F227B
:1001B0006429741AF715741EF711F4197715F41DD4
:1001C00077117419F714741DF710F4187714F41CD0
:1001D00077105F226B29F419F715F41DF7117419C4
:1001E0007715741D7711F418F714F41CF7107418B0
:1001F0007714741C77105F2272297419F715741D17
:10020000F711F4187715F41C77117418F714741C8F
:10021000F710F51B7714F51F77105F227929F41872
:10022000F715F41CF71174187715741C7711F51B6A
:10023000F714F51FF710751B7714751F77105F22E1
:1002400080297418F715741CF711F51B7715F51F25
:100250007711751BF714751FF710F51A7714F51E33
:1002600077105F2287298510F31A0515F31E0511F3
:10027000851400008510731A0515731E0511851469
:1002800000008510F3190515F31D051185140000F4
:10029000851073190515731D05118514000085104F
:1002A000F3180515F31C051185140000851073184B
:1002B0000515731C0511851400008510F41B051528
:1002C000F41F0511851400008510741B0515741F9B
:1002D0000511851400008510F41A0515F41E05118A
:1002E000851400008510741A0515741E05118514F7
:1002F00000008510F4190515F41D05118514000082
:10030000851074190515741D0511851400008510DC
:10031000F4180515F41C05118514000085107418D7
:100320000515741C0511851400008510F51B0515B5
:10033000F51F0511851400008510751B0515751F27
:100340000511851400008510F51A0515F51E051117
:10035000851400008510751A0515751E0511851484
:1003600000008510F5190515F51D0511851400000F
:10037000851075190515751D05118514000085106A
:10038000F5180515F51C0511851400008510751864
:100390000515751C05118514F91CE2290511851038
:1003A000051083160515831205140000051DD629B6
:1003B0000510831605118312831603130C1683127E
:1003C0000313252A791D1C2AFA0105118510000046
:1003D000851483160515831285100519FA178514DF
:1003E0000000851005197A1785140000851005197D
:1003F000FA1685140000851005197A168514000078
:1004000085100519FA1585140000851005197A154F
:100410008514000085100519FA1485140000851054
:1004200005197A1405108316051183128316031318
:100430000C1683120313252A051185100510831647
:1004400003130C1683120313252A83120313981C1B
:100450000F28181218160F28791D302A7A08312A09
:100460007808831203139900831603130C12831266
:1004700003131728700E8300F10E710E090083120A
:1004800003138501860183160313F8308500FF30BE
:100490008600F8309B008130990024309800831248
:1004A00003139030980085018601F601831603132B
:1004B0008B170B178C160C12831203139A2A033016
:1004C0007702031D682A0130F8000130F9000800A6
:1004D00000307702031D712A0630F8000130F90060
:1004E000080002307702031D7A2A0330F800023038
:1004F000F900080001307702031D832A0530F80057
:100500000230F900080077080C390C3C031D8D2AD5
:100510000230F8000230F900080077080439043C82
:10052000031D972A0430F8000230F9000800043057
:06053000F90008009A2A00
:02400E00223F4F
:02401000FC3F73
:00000001FF
